:100000000C9463000C94930A0C94C00A0C948B001B
:100010000C948B000C948B000C948B000C94EC07CC
:100020000C948B000C948B000C948B000C948B0024
:100030000C948B000C948B000C948B000C948B0014
:100040000C94A4130C948B000C9414030C948B004C
:100050000C948B000C948B000C948B000C948B00F4
:100060000C948B000C948B000200000000240027ED
:10007000002A0000000000250028002B00000000DE
:1000800000230026002900040404040404040402DC
:100090000202020202030303030303010204081025
:1000A00020408001020408102001020408102000F2
:1000B0000000070002010000030406000000000029
:1000C00000000000A10411241FBECFEFD8E0DEBF66
:1000D000CDBF12E0A0E0B1E0E0E5F4E402C005909D
:1000E0000D92AA3BB107D9F713E0AAEBB2E001C029
:1000F0001D92A239B107E1F710E0C6ECD0E004C0D0
:100100002297FE010E94881EC43CD107C9F70E94B5
:10011000EF010C9426220C9400000F931F9360EDC6
:1001200077E080E090E00E942C1408E513E0C8011D
:1001300060E071E00E94120560ED77E080E090E001
:100140000E942C14C8010E9482041F910F910895EF
:100150000F931F9386E060E00E941C1508E513E0F2
:10016000C80140E056E960E070E00E94A503C801C4
:100170006BE071E00E941205C80169E171E00E9424
:100180001205C80163E371E00E941205C80161E431
:1001900071E00E941205C8016FE471E00E9412052F
:1001A000C80160E671E00E9412050E948D001F9157
:1001B0000F910895F894FFCF84E061E00E946F15DD
:1001C00083E061E00E946F158AE090E00E94521483
:1001D00084E060E00E946F158AE090E00E94521473
:1001E00083E060E00E946F158AE090E00E94521464
:1001F000089584E060E00E946F158AE090E00E941C
:10020000521483E061E00E946F158AE090E00E9442
:10021000521484E061E00E946F1508958AE090E036
:100220000E94521483E060E00E946F1584E190E028
:100230000E94521483E061E00E946F158AE090E012
:100240000E94521408950F931F938AE090E00E9439
:10025000521400E017E084E00E94A415682F90E09B
:10026000012E02C0880F991F0A94E2F7082B8CE038
:100270000E946F150E940E01115068F70E940E0136
:10028000802F1F910F9108958AE090E00E945214F0
:1002900083E061E00E946F1584E190E00E945214B7
:1002A00083E060E00E946F158AE090E00E945214A3
:1002B00008951F93CF93DF9317E0C82FD0E0BE01BE
:1002C000012E02C0759567950A94E2F7617084E08B
:1002D0000E946F150E944401115088F784E061E08C
:1002E0000E946F150E944401DF91CF911F910895E4
:1002F00084E060E00E941C1583E061E00E946F15BD
:10030000089584E061E00E941C1583E061E00E9492
:100310006F150895EF92FF920F931F938091C5027E
:10032000879588278795F090C602FF0CFF0CFF0C7D
:10033000F82A8091C702F82A8091C9028295880F15
:10034000807E0091CA02000F000F000F082B8091E1
:10035000C802082B9091CB02979599279795809189
:10036000CF028295807F892B9091D102892B909129
:10037000D302990F990F990F982BE090CE02EE0CB3
:10038000E92A9091CC029795992797958091CD0273
:100390008295880F880F807C892B9091D202892BBF
:1003A0001091D002110F110F182B0E9481010E9491
:1003B000DC0088EC0E9459018F2D0E945901802F8A
:1003C0000E9459018E2D0E945901812F0E945901CE
:1003D0000E94F9001F910F91FF90EF9008958F9266
:1003E0009F92AF92BF92CF92DF92EF92FF920F93C4
:1003F0001F93DF93CF93CDB7DEB727970FB6F8944F
:10040000DEBF0FBECDBF0E945C1485E061E00E949C
:100410001C1585E060E00E946F150E94A80082E034
:1004200060E00E941C1583E061E00E941C1586E0DC
:1004300060E00E941C158CE061E00E941C158DE0BC
:1004400061E00E941C158DE061E00E946F1585E05F
:1004500061E00E946F156AEF70E080E090E00E941A
:100460002C140E948A01AAEFEA2EF12C4E01089466
:10047000811C911CF4E0AF2EB12CAC0EBD1EE2E04D
:10048000CE2ED12CCC0EDD1E82E00E94A415019749
:1004900009F0BCC08CE061E00E946F158DE060E067
:1004A0000E946F150E9481010E94DC0089EC0E946D
:1004B000590182E00E94A415892B09F0A7C08DE0A4
:1004C00061E00E946F150E9478010BEB12E00E9420
:1004D0002301F80181938F01F2E0053C1F07B9F772
:1004E0000E9481010E94F9008091BB0289832091C2
:1004F000BD0230E040E050E0542F432F322F22273E
:100500008091BE0290E0A0E0B0E0282B392B4A2B6E
:100510005B2B8091BC0290E0A0E0B0E0877090700F
:10052000A070B070DC0199278827282B392B4A2B23
:100530005B2B2C833D834E835F832091C0022295E9
:1005400026952695237030E08091BF0290E0880FB9
:10055000991F880F991F282B392B3B832A8317C09B
:1005600088E593E00E945E04823029F0833061F0D8
:10057000813069F404C02AEFE22EF12C08C098EE15
:10058000E92E93E0F92E03C082E3E82EF12C88E5F2
:1005900093E00E9433041816190614F386E00E94B3
:1005A000A4152091BA02892B59F1222319F481E074
:1005B0008093BA0288E593E063E771E042E050E09F
:1005C0000E94F30488E593E062E771E041E050E0C7
:1005D0000E94F30488E593E0B40141E050E00E94FA
:1005E000F30488E593E0B50144E050E00E94F30491
:1005F00088E593E0B60142E050E00E94F30406C0B3
:10060000222321F00E948D001092BA02B70180E0EF
:1006100090E00E942C148CE060E00E946F158DE049
:1006200060E00E946F1530CF1F920F920FB60F92AD
:1006300011242F933F934F938F939F93EF93FF93A7
:100640004091C600E0915403F091550331969F010B
:100650002F77307031978091560390915703281768
:10066000390739F0EC52FD4F408330935503209306
:100670005403FF91EF919F918F914F913F912F9153
:100680000F900FBE0F901F9018958F92AF92CF9240
:10069000DF92EF92FF920F931F93DF93CF93CDB72B
:1006A000DEB7FC0189E791E09183808373836283E5
:1006B000558344833783268311870087F386E28638
:1006C000D586C486A68687868D85808B8E85818B10
:1006D0008F85828BCF91DF911F910F91FF90EF90CB
:1006E000DF90CF90AF908F9008958F92AF92CF927E
:1006F000DF92EF92FF920F931F93DF93CF93CDB7CB
:10070000DEB7FC0189E791E0918380837383628384
:10071000558344833783268311870087F386E286D7
:10072000D586C486A68687868D85808B8E85818BAF
:100730008F85828BCF91DF911F910F91FF90EF906A
:10074000DF90CF90AF908F900895EF92FF920F932C
:100750001F938C019A01AB01DC011896ED91FC917D
:10076000199791E0E92EF12CC70152960C9002C026
:10077000880F991F0A94E2F7808360E874E88EE19D
:1007800090E00E94121E215030404040504056954B
:10079000479537952795D8011496ED91FC911597BB
:1007A00030831696ED91FC91179720831A96ED9160
:1007B000FC911B972081C7011E960C901E9702C0CA
:1007C000880F991F0A94E2F7282B20831A96ED913F
:1007D000FC911B972081C7011F960C901F9702C0A8
:1007E000880F991F0A94E2F7282B20831A96ED911F
:1007F000FC911B97808150960C9002C0EE0CFF1C60
:100800000A94E2F78E2980831F910F91FF90EF9059
:100810000895FC01A285B3854C9121E030E0C90127
:10082000068402C0880F991F0A94E2F780958423FA
:100830008C93A285B3854C91C901078402C0880FAF
:10084000991F0A94E2F7809584238C93A285B3853F
:100850008C91008802C0220F331F0A94E2F7209582
:1008600028232C930895DC011296ED91FC911397A7
:10087000E058FF4F2191319180819181281B390BE4
:100880002F773070C9010895DC011296ED91FC912B
:100890001397EE57FF4F2081318192918291E0585A
:1008A000F0408217930719F42FEF3FEF05C0E20FD6
:1008B000F31F8081282F30E0C9010895DC011296D2
:1008C000ED91FC911397DF01AE57BF4F2D913C91F5
:1008D0001197E058FF4F80819181E058F0408217D6
:1008E000930719F42FEF3FEF0BC0E20FF31F808146
:1008F0002F5F3F4F2F7730702D933C93282F30E0A0
:10090000C9010895DC011296ED91FC911397EE5701
:10091000FF4F80819181929382930895FC01A0857D
:10092000B18521898C9190E0022E02C09595879522
:100930000A94E2F780FFF6CF0484F585E02D60830A
:10094000089589E791E0909359038093580384EDCB
:1009500092E090935B0380935A0385EC90E0909330
:100960005D0380935C0384EC90E090935F0380933D
:100970005E0380EC90E0909361038093600381ECD0
:1009800090E0909363038093620386EC90E09093F1
:1009900065038093640384E08093660383E080931F
:1009A000670387E08093680385E08093690381E0B3
:1009B00080936A0308950F931F93CF93DF938C0165
:1009C000EB0109C02196D801ED91FC910190F081D5
:1009D000E02DC801099568816623A1F7DF91CF91C9
:1009E0001F910F910895EF92FF920F931F93CF9352
:1009F000DF938C017B01EA010CC0D7016D917D0171
:100A0000D801ED91FC910190F081E02DC80109958C
:100A10002197209791F7DF91CF911F910F91FF9030
:100A2000EF900895DC01ED91FC910280F381E02DBF
:100A300009950895CF92DF92EF92FF920F931F9343
:100A4000CF93DF936C017B01C0E0D0E00EC0D601F4
:100A5000ED91FC9100811181C701BE010E94B40B90
:100A6000682FC601F80109952196F70184819581C7
:100A7000C817D90760F3DF91CF911F910F91FF90B5
:100A8000EF90DF90CF9008952F923F924F925F9218
:100A90006F927F928F929F92AF92BF92CF92DF928E
:100AA000EF92FF920F931F93DF93CF93CDB7DEB7F3
:100AB000A0970FB6F894DEBF0FBECDBF1C016A0130
:100AC0007B01411551056105710549F440E350E092
:100AD00060E070E020E030E00E94100656C08824FC
:100AE00099245401422E55246624772401E010E015
:100AF0000C0F1D1F080D191DC701B601A30192019E
:100B00000E94121EF80160830894811C911CA11C94
:100B1000B11CC701B601A30192010E94121EC901B6
:100B2000DA016C017D01C114D104E104F104F1F694
:100B300081E0E82EF12CEC0EFD1EE80CF91C3E01C4
:100B40000894611C711CD501C4010197A109B10968
:100B50006C01C818D90816C0F601EE0DFF1D4081C2
:100B60004A3010F4405D01C0495C552747FD50955F
:100B7000652F752FC10120E030E00E941006089417
:100B8000E108F1086E147F0439F7A0960FB6F894C7
:100B9000DEBF0FBECDBFCF91DF911F910F91FF90B0
:100BA000EF90DF90CF90BF90AF909F908F907F900D
:100BB0006F905F904F903F902F900895DC0121152A
:100BC000310541F4ED91FC910190F081E02D642F0D
:100BD000099508950E9444050895EF92FF920F939E
:100BE0001F939A017B0100E010E0B801A7010E9469
:100BF000DE051F910F91FF90EF900895EF92FF9205
:100C00000F931F939A01E62EFF2400E010E0B80135
:100C1000A7010E94DE051F910F91FF90EF900895AC
:100C2000EF92FF920F931F93CF93DF93EC017A0122
:100C30008B012115310541F4E881F9810190F081A2
:100C4000E02D642F09951BC02A303105B1F477FFE0
:100C500010C04DE250E060E070E020E030E00E9423
:100C6000100610950095F094E094E11CF11C011D14
:100C7000111DCE01B801A7012AE00E944405DF91B1
:100C8000CF911F910F91FF90EF900895EF92FF92F7
:100C90000F931F937B019A010027F7FC0095102FFB
:100CA000B801A7010E9410061F910F91FF90EF90CD
:100CB0000895EF92FF920F931F93E62E9A01FF245F
:100CC000E7FCF0940F2D1F2DB801A7010E9410061C
:100CD0001F910F91FF90EF9008950F931F938C0138
:100CE0004DE050E060E070E020E030E00E9410064F
:100CF000C8014AE050E060E070E020E030E00E948F
:100D000010061F910F9108950F931F938C010E945D
:100D1000DE05C8010E946D061F910F910895CF92C4
:100D2000DF92EF92FF920F931F938C019A016B0158
:100D3000EE24FF24B701A6010E94DE05C8010E942F
:100D40006D061F910F91FF90EF90DF90CF90089567
:100D5000CF92DF92EF92FF920F931F938C019A0133
:100D6000C62EDD24EE24FF24B701A6010E94DE0575
:100D7000C8010E946D061F910F91FF90EF90DF90C8
:100D8000CF9008950F931F938C010E941205C80104
:100D90000E946D061F910F9108950F931F938C0170
:100DA0000E941A05C8010E946D061F910F910895B7
:100DB0000F931F938C010E941006C8010E946D06BC
:100DC0001F910F910895CF92DF92EF92FF920F93B0
:100DD0001F938C016B019A01EE24D7FCE094FE2C4A
:100DE000B701A6010E941006C8010E946D061F915E
:100DF0000F91FF90EF90DF90CF900895CF92DF9208
:100E0000EF92FF920F931F938C01C62E9A01DD245F
:100E1000C7FCD094ED2CFD2CB701A6010E94100652
:100E2000C8010E946D061F910F91FF90EF90DF9017
:100E3000CF9008959F92AF92BF92CF92DF92EF92A0
:100E4000FF920F931F93CF93DF93EC017A018B01F5
:100E5000922ECB01BA0120E030E040E050E00E9449
:100E6000A31A88236CF4CE014DE250E060E070E0FC
:100E700020E030E00E94100617FB109517F910953E
:100E800020E030E040E05FE3AA240BC0CA01B901D2
:100E900020E030E040E251E40E94C7199B01AC0120
:100EA000A394A91498F3C801B7010E94A0185B018C
:100EB0006C010E94F7167B018C01CE01B801A701DD
:100EC0002AE030E00E94DE05992029F0CE0169E990
:100ED00071E00E941205C801B7010E94851B9B01A9
:100EE000AC01C601B5010E946F1822C020E030E0BD
:100EF00040E251E40E94CD187B018C010E94311B1D
:100F00005B016C01CC24B7FCC094DC2CCE01B60193
:100F1000A5012AE030E00E941006C601B5010E943A
:100F2000D31A9B01AC01C801B7010E946F189A94B3
:100F30009920E1F6DF91CF911F910F91FF90EF90F3
:100F4000DF90CF90BF90AF909F9008950E941A07B6
:100F500008950F931F938C010E941A07C8010E94E5
:100F60006D061F910F910895813041F0813018F086
:100F70008230D1F409C010926E00089580916F0004
:100F80008D7F80936F000895809170008D7F809396
:100F9000700081E08093B0008091B100887F846010
:100FA0008093B1001092B30008951F93182F809181
:100FB000A501811711F09FEF06C0E8E6F0E09491DB
:100FC0008FEF8093A501892F0E94B407812F60E0E5
:100FD0000E946F151F9108951F920F920FB60F92E6
:100FE00011242F933F934F935F936F937F938F932E
:100FF0009F93AF93BF93EF93FF9380917903909169
:101000007A03A0917B03B0917C030097A105B10501
:1010100051F1E0917D03F0917E03808190917F03F7
:10102000892780838091790390917A03A0917B0333
:10103000B0917C03181619061A061B06C4F4809199
:10104000790390917A03A0917B03B0917C0301977F
:10105000A109B1098093790390937A03A0937B034C
:10106000B0937C0304C08091A5010E94D507FF9135
:10107000EF91BF91AF919F918F917F916F915F9110
:101080004F913F912F910F900FBE0F901F90189589
:101090002F923F925F926F927F928F929F92AF9228
:1010A000BF92CF92DF92EF92FF920F931F93DF9345
:1010B000CF9300D000D0CDB7DEB7A82F1B01298376
:1010C0003A834B835C838091A5018A1721F4E8E67B
:1010D000F0E0549082C08F3F09F0D9C1A093A501E0
:1010E000E8E6F0E054902FEF521609F4D0C181E009
:1010F000581639F192E0591609F449C0552009F003
:101100006CC014BC15BC84B5826084BD85B581609B
:1011100085BD2A2F30E0F901E957FF4FE491F0E057
:10112000EE0FFF1FED58FF4F859194919093700340
:1011300080936F0325563F4FF9018491809371038B
:101140004EC01092800010928100809181008860D2
:1011500080938100809181008160809381002A2F9B
:1011600030E0F901E957FF4FE491F0E0EE0FFF1F87
:10117000ED58FF4F85919491909377038093760378
:1011800025563F4FF90184918093780328C010922F
:10119000B0001092B1008091B00082608093B000E6
:1011A0008091B10081608093B1002A2F30E0F90175
:1011B000E957FF4FE491F0E0EE0FFF1FED58FF4FAE
:1011C0008591949190937E0380937D0325563F4FA4
:1011D000F901849180937F0302C057FC58C18A2F84
:1011E00061E00E941C15552021F0F2E05F1609F025
:1011F000BDC031018824992460E079E08DE390E05E
:10120000A40193010E94121E59016A018601750111
:101210000894E108F108010911092FEFE216F10421
:101220000105110509F008F498C060E271EA87E051
:1012300090E0A40193010E94121E79018A01089492
:10124000E108F1080109110982E05816C1F49FEF85
:10125000E916F1040105110509F008F483C068E4FA
:1012600078EE81E090E0A40193010E94121E7901C2
:101270008A010894E108F1080109110983E0AFEF40
:10128000EA16F1040105110509F008F467C064E2EB
:1012900074EF80E090E0A40193010E94121E790196
:1012A0008A010894E108F10801091109552011F497
:1012B00083E01DC0B2E05B1611F084E018C0EFEFD0
:1012C000EE16F1040105110509F008F4DEC062E133
:1012D0007AE780E090E0A40193010E94121E790158
:1012E0008A010894E108F1080109110985E0FFEF7E
:1012F000EF16F1040105110589F180F169E07DE344
:1013000080E090E0A40193010E94121E79018A01FD
:101310000894E108F10801091109552011F086E04F
:1013200001C084E02FEFE216F10401051105B1F0D0
:10133000A8F0860175019AE016950795F794E79451
:101340009A95D1F70894E108F1080109110955208F
:1013500011F087E008C085E003C081E0552019F452
:1013600085BD3AC082E08093B10036C05101CC24E3
:10137000DD2460E079E08DE390E0A60195010E9414
:10138000121E79018A010894E108F1080109110986
:1013900080E0E81680E0F80681E0080780E01807A2
:1013A00010F491E010C064E274EF80E090E0A601D8
:1013B00095010E94121E79018A010894E108F10842
:1013C0000109110993E0A1E05A1631F480918100DE
:1013D000887F982B9093810089819A81AB81BC8111
:1013E0000097A105B10529F48FEF9FEFAFEFBFEF95
:1013F00013C0220C331CB10180E090E029813A81B6
:101400004B815C810E94F31D28EE33E040E050E008
:101410000E94121EC901DA01E1E05E16A1F0F2E0BD
:101420005F1619F1552099F5E7BC80936B039093F3
:101430006C03A0936D03B0936E0380916E00826085
:1014400080936E0024C0F0928900E092880080931F
:10145000720390937303A0937403B0937503809108
:101460006F00826080936F0012C0E092B30080939F
:10147000790390937A03A0937B03B0937C038091CC
:10148000700082608093700002C084E06CCF0F9087
:101490000F900F900F90CF91DF911F910F91FF90C0
:1014A000EF90DF90CF90BF90AF909F908F907F9004
:1014B0006F905F903F902F900895823000F5E82F55
:1014C000F0E0EE0FFF1FE058FC4F7183608388232C
:1014D00019F08130A1F408C0809169008C7F842BC1
:1014E00080936900E89A089580916900440F551F20
:1014F000440F551F837F842B80936900E99A0895D8
:10150000823080F4882319F0813021F402C0E898F9
:1015100001C0E998E82FF0E0EE0FFF1FE058FC4F04
:101520001182108208951F920F920FB60F9211240C
:101530002F933F934F935F936F937F938F939F93DB
:10154000AF93BF93EF93FF938091800390918103BA
:10155000892B29F0E0918003F09181030995FF9197
:10156000EF91BF91AF919F918F917F916F915F911B
:101570004F913F912F910F900FBE0F901F90189594
:101580001F920F920FB60F9211242F933F934F93F8
:101590005F936F937F938F939F93AF93BF93EF93DB
:1015A000FF938091820390918303892B29F0E0912E
:1015B0008203F09183030995FF91EF91BF91AF9161
:1015C0009F918F917F916F915F914F913F912F915B
:1015D0000F900FBE0F901F9018952F923F924F9231
:1015E0005F926F927F928F929F92AF92BF92CF92B3
:1015F000DF92EF92FF920F931F93DF93CF93CDB7BC
:10160000DEB73B014C0119012A016D897E898F8962
:10161000988D6A197B098C099D09621A730A840ADC
:10162000950AA40193010E94F31DE218F30804092E
:101630001509A80197010E94341E2A0D3B1D4C1D5F
:101640005D1DB901CA01CF91DF911F910F91FF90EC
:10165000EF90DF90CF90BF90AF909F908F907F9052
:101660006F905F904F903F902F900895089570E095
:10167000382F20E0622B732BCB010895EF92FF925D
:101680000F931F937B018C016115710581059105F5
:1016900029F420E030E040E050E00BC00E94E41F5D
:1016A000A80197010E94341EAC01CB01DA019C0114
:1016B000AD01B901CA011F910F91FF90EF900895FC
:1016C000EF92FF920F931F937B018C0162177307B8
:1016D0008407950764F4261B370B480B590BCA0186
:1016E000B9010E943E0BE60EF71E081F191FB70135
:1016F000C8011F910F91FF90EF900895009729F076
:10170000BC0180E090E00E94E91F0895FC01019077
:10171000F081E02DE60FF71F80810895DC01ED9147
:10172000FC911197309751F014968D919C911597DB
:101730006817790718F4E60FF71F40830895FC0136
:101740009B01848195816817790728F460817181F4
:101750006115710529F41092840364E873E002C0F6
:10176000620F731FCB010895FC010190F081E02D01
:10177000E60FF71F80810895FC01808191810E940E
:10178000C02008950F931F93CF93DF93FC018B012B
:1017900041155105A1F06115710589F0848195818C
:1017A000EA0121978C179D0708F4EC016081718193
:1017B000C801AE010E943C21C00FD11F1882DF91E9
:1017C000CF911F910F9108950F931F93CF93DF93A4
:1017D000FC018B0141155105A1F06115710589F0DE
:1017E00084819581EA0121978C179D0708F4EC010B
:1017F00060817181C801AE010E943C21C00FD11FE0
:101800001882DF91CF911F910F9108950F931F932D
:101810008C01FC01808191810E94391FF8011382A3
:101820001282158214821F910F910895FC01DB0131
:1018300014962D913C91159784819581821B930B71
:101840008417950710F480E00895808191816D914F
:101850007C91840F951FA9010E942E219C0180E09C
:10186000232B09F481E00895FC01DB0124813581FB
:1018700014968D919C9115972817390710F480E0E4
:101880000895CF0140E050E00E94160C0895DF92C9
:10189000EF92FF920F931F93CF93DF93EC018C8114
:1018A0009D8148175907C8F47A010894E11CF11C7E
:1018B000E881F981EE0DFF1DD08010820881198129
:1018C000772767FD7095C8010E944B219C010E0D82
:1018D0001F1DF801D082009719F4EFEFFFEF05C04C
:1018E00088819981F901E81BF90BCF01DF91CF9134
:1018F0001F910F91FF90EF90DF900895FC014481BC
:101900005581415050400E94470C0895CF93DF937A
:10191000FC01DB01848195814817590760F4C0817F
:10192000D1816D917C91CE01840F951F0E9456212B
:101930009C01009719F42FEF3FEF02C02C1B3D0BC9
:10194000C901DF91CF91089540E050E00E94860CDC
:101950000895CF93DF93FC0184819581481759073F
:1019600068F4C081D181772767FD7095CE01840F1F
:10197000951F0E9413219C01009719F42FEF3FEF50
:1019800002C02C1B3D0BC901DF91CF91089540E0AF
:1019900050E00E94A90C0895DC01FB0114962D91E2
:1019A0003C911597848195812817390711F080E0C3
:1019B0000895608171818D919C910E941E219C01EE
:1019C00080E0232B09F481E00895FC01DB012481F0
:1019D000358114968D919C9115972817390710F42D
:1019E00080E00895281B390B808191816D917C9155
:1019F000820F931F0E941E219C0180E0232B09F47B
:101A000081E00895DC01FB01608171818D919C91E1
:101A10000E941E21292F332727FD309520953095D0
:101A20002227330F221F3327C9010895DC01FB0150
:101A3000608171818D919C910E941E2140E050E057
:101A40001816190614F041E050E0CA010895DC01AF
:101A5000FB01608171818D919C910E941E2140E06B
:101A600050E01816190614F441E050E0CA01089538
:101A7000DC01FB01608171818D919C910E941E218E
:101A8000292F332727FD30952227330F221F332795
:101A9000C9010895DC01FB0114962D913C91159725
:101AA000848195812817390751F4608171818D9166
:101AB0009C910E941E219C0180E0232B09F081E073
:101AC00090E00895DC01FB0114962D913C9115974F
:101AD000848195812817390711F080E00BC060815F
:101AE00071818D919C910E941E219C0180E0232B8D
:101AF00009F481E090E00895FC01DB016D917C9197
:101B0000808191810E941E2108950F931F93CF938E
:101B1000DF93EC018B01FB01648175818C819D81D8
:101B2000680F791F7D836C838A819B818617970755
:101B3000B8F46F5F7F4F888199810E94F21F4C81BA
:101B40005D81009729F0998388835B834A8308C06D
:101B5000F80184819581481B590B5D834C8307C034
:101B6000F80160817181888199810E940821CE01EC
:101B7000DF91CF911F910F9108950E94850D0895D7
:101B8000CF93DF93EC01CB017B836A8301960E94A4
:101B90008C1E99838883009721F41B821A821D82F0
:101BA0001C82DF91CF9108950F931F93CF93DF9302
:101BB000EC018B018617970709F1FB012481358120
:101BC0008C819D818217930750F4888199810E94AE
:101BD000391FF80164817581CE010E94C00D2881F2
:101BE00039812115310551F0F801848195819D835A
:101BF0008C8360817181C9010E942721CE01DF9110
:101C0000CF911F910F9108951F93CF93DF93EC0114
:101C1000162F81E090E09D838C83CE0161E070E01F
:101C20000E94C00DE881F981309721F01083E8818E
:101C3000F9811182DF91CF911F9108951F93CF9366
:101C4000DF93EC01162F81E090E09D838C83CE0121
:101C500061E070E00E94C00DE881F981309721F0C9
:101C60001083E881F9811182DF91CF911F9108954E
:101C70001F93CF93DF93EC01162F81E090E09D83BB
:101C80008C83CE0161E070E00E94C00DE881F98193
:101C9000309721F01083E881F9811182DF91CF9193
:101CA0001F9108951F93CF93DF93EC01162F81E0CE
:101CB00090E09D838C83CE0161E070E00E94C00DB6
:101CC000E881F981309721F01083E881F981118250
:101CD000DF91CF911F9108950F931F93CF93DF93BF
:101CE0008C01EB016C817D81FC01758364830E9412
:101CF000C00DF80180819181009721F06881798180
:101D00000E942721DF91CF911F910F9108950F938A
:101D10001F93CF93DF938C01EB016C817D81FC01DC
:101D2000758364830E94C00DF801808191810097C2
:101D300021F0688179810E942721DF91CF911F9145
:101D40000F910895EF92FF920F931F93DF93CF931C
:101D5000CDB7DEB7A1970FB6F894DEBF0FBECDBFEB
:101D60008C01CB01BA017E010894E11CF11CA70192
:101D70002AE030E00E94DA21F70101900020E9F723
:101D80003197EE19FF09D8011596FC93EE9314973D
:101D9000C801BF010E94C00DF801808191810097A8
:101DA00019F0B7010E942721A1960FB6F894DEBF63
:101DB0000FBECDBFCF91DF911F910F91FF90EF909C
:101DC0000895EF92FF920F931F93DF93CF93CDB7B8
:101DD000DEB7A1970FB6F894DEBF0FBECDBF8C0162
:101DE000CB01BA017E010894E11CF11CA7012AE095
:101DF00030E00E94DA21F70101900020E9F73197E5
:101E0000EE19FF09D8011596FC93EE931497C801BB
:101E1000BF010E94C00DF80180819181009719F0E7
:101E2000B7010E942721A1960FB6F894DEBF0FBE1E
:101E3000CDBFCF91DF911F910F91FF90EF9008954B
:101E4000EF92FF920F931F93DF93CF93CDB7DEB73F
:101E5000A1970FB6F894DEBF0FBECDBF8C019A01DB
:101E600080E090E07E010894E11CF11CA7010E9433
:101E7000DA21F70101900020E9F73197EE19FF0907
:101E8000D8011596FC93EE931497C801BF010E94E8
:101E9000C00DF80180819181009719F0B7010E946F
:101EA0002721A1960FB6F894DEBF0FBECDBFCF910C
:101EB000DF911F910F91FF90EF900895EF92FF92A5
:101EC0000F931F93DF93CF93CDB7DEB7A1970FB6D4
:101ED000F894DEBF0FBECDBF8C019A0180E090E088
:101EE0007E010894E11CF11CA7010E94DA21F70190
:101EF00001900020E9F73197EE19FF09D8011596F6
:101F0000FC93EE931497C801BF010E94C00DF80125
:101F100080819181009719F0B7010E942721A19635
:101F20000FB6F894DEBF0FBECDBFCF91DF911F91EA
:101F30000F91FF90EF9008950F931F93CF93DF932E
:101F40008C01EB016115710511F4C6EAD1E0FE01C7
:101F500001900020E9F73197EC1BFD0BD801159695
:101F6000FC93EE931497C801BF010E94C00DF801C5
:101F700080819181009719F0BE010E942721DF9195
:101F8000CF911F910F910895AF92BF92CF92DF92A0
:101F9000EF92FF920F931F93CF93DF93B82EA92E4A
:101FA0006B01C82FD92FFB0160817181CE010E9486
:101FB0009C0FEE24FF2410C0088119810E0D1F1DF7
:101FC000F8018081992787FD90950E94F720F801FC
:101FD00080830894E11CF11CF60184819581E81648
:101FE000F90650F38B2D9A2DDF91CF911F910F9110
:101FF000FF90EF90DF90CF90BF90AF900895AF9299
:10200000BF92CF92DF92EF92FF920F931F93CF93E5
:10201000DF93B82EA92E6B01C82FD92FFB01608149
:102020007181CE010E949C0FEE24FF2410C0088114
:1020300019810E0D1F1DF8018081992787FD90954C
:102040000E94EF20F80180830894E11CF11CF60146
:1020500084819581E816F90650F38B2D9A2DDF9136
:10206000CF911F910F91FF90EF90DF90CF90BF9095
:10207000AF900895EF92FF920F931F93DF93CF934A
:10208000CDB7DEB72C970FB6F894DEBF0FBECDBF2D
:10209000FC017B018617970711F401E029C0248118
:1020A0003581DB0114968D919C911597281739077E
:1020B00011F000E01DC0CE010196BF010E94FF0F8C
:1020C00009811A81CE010796B7010E94FF0F6F8127
:1020D0007885C8010E941E2100E0009709F401E004
:1020E000CE0107960E94060CCE0101960E94060CB6
:1020F000802F2C960FB6F894DEBF0FBECDBFCF91C8
:10210000DF911F910F91FF90EF900895CF92DF9292
:10211000EF92FF921F93CF93DF936C017B01B90184
:102120002417350710F4BA01A901D70114968D912F
:102130009C911597EB018617970708F4EC01D701DE
:10214000ED91FC911197EC0FFD1F108110826D91A4
:102150007C91640F751FC6010E949C0FD701ED9101
:10216000FC91EC0FFD1F1083C601DF91CF911F91F1
:10217000FF90EF90DF90CF9008950F931F938C0105
:10218000FB01248135810E948610C8011F910F91A7
:1021900008958F929F92AF92BF92CF92DF92EF926B
:1021A000FF920F931F93DF93CF9300D000D000D006
:1021B000CDB7DEB75C016B01DB0114968D919C916C
:1021C00015970097A1F101974817590780F1F5017C
:1021D000848195814817590750F5ED91FC91008154
:1021E0007A014E010894811C911C1FC0D501ED910C
:1021F000FC91EE0DFF1D80818017A1F4F601248172
:1022000035812E0D3F1DC401B501A7010E94861026
:10221000C401B6010E94CC0C182FC4010E94060C08
:10222000112341F40894E108F108F7FEDFCFEE2412
:10223000EA94FE2CC70126960FB6F894DEBF0FBEB7
:10224000CDBFCF91DF911F910F91FF90EF90DF9065
:10225000CF90BF90AF909F908F900895FC01DB01CD
:102260004481558114968D919C911597481B590B6B
:10227000CF010E94C9100895AF92BF92CF92DF9212
:10228000EF92FF920F931F93DF93CF9300D000D074
:1022900000D0CDB7DEB75C018B01DB016D917C9185
:1022A0006115710521F4B8010E946C0E42C0CE0187
:1022B00001960E949C0FF801E480F580CC24DD2477
:1022C00010C0D801ED91FC91EC0DFD1D8081992786
:1022D00087FD90950E94E720892B31F00894C11C5E
:1022E000D11CCE14DF0468F3ED80FE800DC0D80150
:1022F000ED91FC91EE0DFF1D8081992787FD909552
:102300000E94E720892B31F00894E108F108CE14EF
:10231000DF0468F30894E11CF11CC5018E010F5F16
:102320001F4FB801A60197010E948610C8010E94A4
:10233000060CC50126960FB6F894DEBF0FBECDBFC2
:10234000CF91DF911F910F91FF90EF90DF90CF9091
:10235000BF90AF9008952F923F924F925F926F92ED
:102360007F928F929F92AF92BF92CF92DF92EF9225
:10237000FF920F931F93DF93CF93CDB7DEB768978C
:102380000FB6F894DEBF0FBECDBF3C01FB012A01A2
:102390001901608171816115710521F4BF010E94ED
:1023A0006C0E5AC07E010894E11CF11CC7010E940A
:1023B0009C0F8E01095F1F4FC80166EA71E00E9401
:1023C0009C0FD02EC12E3DE0832E912C8C0E9D1E95
:1023D00023E1A22EB12CAC0EBD1E24C0C401B70156
:1023E00040E050E098010E9486108D2D9C2DB40194
:1023F0000E94850DC4010E94060C8D2D9C2DB101FB
:102400000E94850DF20144815581400F511FC50185
:10241000B7010E94BD10C701B5010E94D40DC501CE
:102420000E94060CC701B2010E94A40C8C01FFEFB0
:102430008F3F9F0799F68D2D9C2DB7010E94850D2A
:10244000C3016D2D7C2D0E946C0E8D2D9C2D0E9444
:10245000060CC7010E94060CC30168960FB6F894DB
:10246000DEBF0FBECDBFCF91DF911F910F91FF90C7
:10247000EF90DF90CF90BF90AF909F908F907F9024
:102480006F905F904F903F902F900895DF92EF9262
:10249000FF920F931F93DF93CF9300D000D000D013
:1024A000CDB7DEB77C01FB01142FD22E6081718184
:1024B0006115710521F4BF010E946C0E1CC0CE0194
:1024C00001960E949C0F89819A81012F112707FD97
:1024D000109501C0D082B8010E941321FC01009721
:1024E000C9F7C7018E010F5F1F4FB8010E946C0E24
:1024F000C8010E94060CC70126960FB6F894DEBFED
:102500000FBECDBFCF91DF911F910F91FF90EF9044
:10251000DF9008950F931F93CF93DF938C01EB010E
:102520006115710511F4C6EAD1E0FE0101900020A9
:10253000E9F73197EC1BFD0BD8011596FC93EE9350
:102540001497C801BF010E94C00DF80180819181DC
:10255000009719F0BE010E942721DF91CF911F91B2
:102560000F910895EF92FF920F931F93DF93CF93F4
:10257000CDB7DEB7A1970FB6F894DEBF0FBECDBFC3
:102580008C01CB01BA017E010894E11CF11CA7016A
:102590000E949121F70101900020E9F73197EE198F
:1025A000FF09D8011596FC93EE931497C801BF015B
:1025B0000E94C00DF80180819181009719F0B70148
:1025C0000E942721A1960FB6F894DEBF0FBECDBFA3
:1025D000CF91DF911F910F91FF90EF900895EF92AF
:1025E000FF920F931F93DF93CF93CDB7DEB7A197E1
:1025F0000FB6F894DEBF0FBECDBF8C01CB01BA0180
:102600007E010894E11CF11CA7010E949121F701B1
:1026100001900020E9F73197EE19FF09D8011596CE
:10262000FC93EE931497C801BF010E94C00DF801FE
:1026300080819181009719F0B7010E942721A1960E
:102640000FB6F894DEBF0FBECDBFCF91DF911F91C3
:102650000F91FF90EF900895EF92FF920F931F93C9
:10266000DF93CF93CDB7DEB7A1970FB6F894DEBF57
:102670000FBECDBF8C01CB017E010894E11CF11C83
:10268000B7010E947021F70101900020E9F731970E
:10269000EE19FF09D8011596FC93EE931497C80123
:1026A000BF010E94C00DF80180819181009719F04F
:1026B000B7010E942721A1960FB6F894DEBF0FBE86
:1026C000CDBFCF91DF911F910F91FF90EF900895B3
:1026D000EF92FF920F931F93DF93CF93CDB7DEB7A7
:1026E000A1970FB6F894DEBF0FBECDBF8C01CB0112
:1026F0007E010894E11CF11CB7010E947021F701D2
:1027000001900020E9F73197EE19FF09D8011596DD
:10271000FC93EE931497C801BF010E94C00DF8010D
:1027200080819181009719F0B7010E942721A1961D
:102730000FB6F894DEBF0FBECDBFCF91DF911F91D2
:102740000F91FF90EF9008951F920F920FB60F9286
:1027500011242F933F934F935F936F937F938F93A6
:102760009F93AF93BF932091890330918A03409147
:102770008B0350918C0370918D03DA01C90102968D
:10278000A11DB11D672F6A5F6D3730F06D57DA01FB
:10279000C9010396A11DB11D60938D038093890328
:1027A00090938A03A0938B03B0938C03809185034D
:1027B00090918603A0918703B09188030196A11D93
:1027C000B11D8093850390938603A0938703B093F4
:1027D0008803BF91AF919F918F917F916F915F918E
:1027E0004F913F912F910F900FBE0F901F90189512
:1027F0008FB7F8942091890330918A0340918B031D
:1028000050918C038FBFB901CA0108959FB7F89406
:10281000209185033091860340918703509188036E
:1028200086B5A89B06C08F3F21F02F5F3F4F4F4FCB
:102830005F4F9FBF542F432F322F2227280F311D68
:10284000411D511D83E0220F331F441F551F8A95E0
:10285000D1F7B901CA010895EF92FF920F931F9328
:10286000CF93DF937B018C010E940614EB010EC015
:102870000E9406146C1B7D0B685E7340C8F30894BD
:10288000E108F10801091109C851DC4FE114F10414
:102890000105110569F7DF91CF911F910F91FF900D
:1028A000EF900895019739F0019729F0880F991F4B
:1028B00001970197F1F70895789484B5826084BDFB
:1028C00084B5816084BD85B5826085BD85B5816034
:1028D00085BDEEE6F0E0808181608083E1E8F0E094
:1028E0001082808182608083808181608083E0E8C3
:1028F000F0E0808181608083E1EBF0E080818460A2
:102900008083E0EBF0E0808181608083EAE7F0E0A3
:102910008081846080838081826080838081816007
:1029200080838081806880831092C10008958093A5
:10293000A7010895982F8E3008F09E5097708091CF
:10294000A7018295880F880F807C892B80937C005B
:1029500080917A00806480937A0080917A0086FD6D
:10296000FCCF2091780040917900942F80E030E0F6
:10297000282B392BC90108951F93CF93DF93182F6C
:10298000EB0161E00E941C15209709F44AC0CF3F7B
:10299000D10509F449C0E12FF0E0E155FF4F8491E2
:1029A0008330C1F0843028F4813051F08230B1F5A9
:1029B0000CC0863019F1873049F1843079F514C0A4
:1029C00084B5806884BDC7BD33C084B5806284BDD2
:1029D000C8BD2EC080918000806880938000D09315
:1029E0008900C093880024C0809180008062809319
:1029F0008000D0938B00C0938A001AC08091B000F1
:102A000080688093B000C093B30012C08091B00082
:102A100080628093B000C093B4000AC0C038D10572
:102A20001CF4812F60E002C0812F61E00E946F15CD
:102A3000DF91CF911F910895482F50E0CA0185562C
:102A40009F4FFC01249149575F4FFA0184918823DD
:102A5000C1F0E82FF0E0EE0FFF1FE759FF4FA591FF
:102A6000B491662341F49FB7F8948C91209582230A
:102A70008C939FBF08959FB7F8948C91822B8C9371
:102A80009FBF0895833071F0843028F48130A1F025
:102A9000823021F514C08630B1F08730D1F0843017
:102AA000E9F404C0809180008F7703C0809180009A
:102AB0008F7D80938000089584B58F7702C084B5A0
:102AC0008F7D84BD08958091B0008F778093B00092
:102AD00008958091B0008F7D8093B0000895FF929B
:102AE0000F931F93F62E482F50E0CA0181559F4F38
:102AF000FC012491CA0185569F4FFC01149149574E
:102B00005F4FFA0104910023D9F0222319F0822F9C
:102B10000E944215E02FF0E0EE0FFF1FED58FF4F2F
:102B2000A591B491FF2031F49FB7F8948C91109542
:102B3000812304C09FB7F8948C91812B8C939FBF05
:102B40001F910F91FF9008950F931F93482F50E00E
:102B5000CA0181559F4FFC012491CA0185569F4FA0
:102B6000FC01049149575F4FFA011491112319F4A4
:102B700020E030E015C0222319F0822F0E94421578
:102B8000812F90E0880F991F83589F4FFC01A591DA
:102B9000B4918C9120E030E0802311F021E030E00E
:102BA000C9011F910F9108958F929F92AF92BF928A
:102BB000CF92DF92EF92FF920F931F93CF93DF9309
:102BC000A82FB0E0CD0185569F4FFC018490A957F6
:102BD000BF4FFD01D490662311F4992401C0982CB5
:102BE000CA01B90120E43FE140E050E00E94F31D3A
:102BF00020E83EE340E050E00E94121E79018A0185
:102C00006D2D70E0660F771F63587F4FAA24BB2499
:102C10006501FB01A591B4910BC0AE14BF04C006C1
:102C2000D10609F44FC00894A11CB11CC11CD11CD1
:102C30008C918821891589F30CC0AE14BF04C0069D
:102C4000D10609F43FC00894A11CB11CC11CD11CC1
:102C500003C0FB01A591B4918C918821891569F776
:102C600020E030E040E050E0FB01C591D4910FC07E
:102C7000DA01C9018A0D9B1DAC1DBD1D8E159F0576
:102C8000A007B107F9F02F5F3F4F4F4F5F4F88818B
:102C90008821891569F3CA01B90128E032E540E0CD
:102CA00050E00E94F31D6058714C8F4F9F4F20E4FD
:102CB0003FE140E050E00E94121EC901DA019C0190
:102CC000AD0104C020E030E040E050E0B901CA01AD
:102CD000DF91CF911F910F91FF90EF90DF90CF90F8
:102CE000BF90AF909F908F900895BF92CF92DF9248
:102CF000EF92FF920F931F93CF93DF93E82EF62E60
:102D0000B42EC7E0D0E0022F10E087E0C82ED12C0F
:102D1000BB2059F4B6016C1B7D0BC80102C0959510
:102D200087956A95E2F7BC0107C0B8010C2E02C076
:102D3000759567950A94E2F761708E2D0E946F1564
:102D40008F2D61E00E946F158F2D60E00E946F153E
:102D500021979FEFCF3FD907D9F6DF91CF911F91F0
:102D60000F91FF90EF90DF90CF90BF900895CF929A
:102D7000DF92EF92FF920F931F93CF93DF93F82E82
:102D8000062FE42E10E0C7E0D0E097E0C92ED12C4A
:102D9000802F61E00E946F15EE2061F48F2D0E945C
:102DA000A41596012C1B3D0B02C0880F991F2A9574
:102DB000E2F709C08F2D0E94A4150C2E02C0880FC7
:102DC000991F0A94E2F7182B802F60E00E946F157C
:102DD00021978FEFCF3FD807D9F6812FDF91CF9181
:102DE0001F910F91FF90EF90DF90CF900895EF9299
:102DF000FF920F931F937B018C0120E030E040E0B5
:102E00005FE40E94731A88238CF0C801B70120E0A8
:102E100030E040E05FE40E946F180E94311B9B018C
:102E2000AC01205030404040504806C0C801B701B6
:102E30000E94311B9B01AC01B901CA011F910F9186
:102E4000FF90EF900895A0E0B0E0E9E2F7E10C9484
:102E50004F1EDC012B01FA019C91923008F439C11C
:102E6000EB018881823008F433C1943069F48430F6
:102E700009F02FC111969C9111978981981709F437
:102E800028C1A8EAB1E025C1843009F421C182300B
:102E9000A9F4923009F01DC19A01AD0188E0EA0160
:102EA0000990AE01E90109929E018150C1F7E2014A
:102EB000898111969C918923818308C1923009F4FC
:102EC00007C112962D903C901397EB018A819B814C
:102ED0001496AD90BD90CD90DC901797EC80FD805E
:102EE0000E811F819101281B390BB90137FF04C0E6
:102EF00066277727621B730B603271050CF061C087
:102F0000121613066CF537014801062E04C096947C
:102F10008794779467940A94D2F721E030E040E0F8
:102F200050E004C0220F331F441F551F6A95D2F78B
:102F300021503040404050402E213F21402351231A
:102F4000211531054105510521F021E030E040E037
:102F500050E079018A01E628F728082919293CC0A0
:102F6000232BD1F1260E371E35014601062E04C053
:102F700096948794779467940A94D2F721E030E08E
:102F800040E050E004C0220F331F441F551F6A95D4
:102F9000D2F721503040404050402A213B214C2163
:102FA0005D21211531054105510521F021E030E079
:102FB00040E050E059016A01A628B728C828D9285E
:102FC0000BC0821593052CF01C01AA24BB246501BB
:102FD00003C0EE24FF24870111969C91D201119623
:102FE0008C91981709F445C0992339F0A8019701ED
:102FF0002A193B094C095D0906C0A60195012E1945
:103000003F09400B510B57FD08C0118233822282C9
:1030100024833583468357831DC081E081833382B7
:10302000228288279927DC01821B930BA40BB50B06
:1030300084839583A683B7830DC0220F331F441F5B
:10304000551F24833583468357838281938101975B
:10305000938382832481358146815781DA01C901B6
:103060000197A109B1098F5F9F4FAF4FBF4328F36D
:103070000BC0918333822282EA0CFB1C0C1D1D1DA8
:10308000E482F5820683178383E08083248135817F
:103090004681578157FF1AC0C901AA2797FDA095FD
:1030A000BA2F81709070A070B07056954795379583
:1030B0002795822B932BA42BB52B84839583A683F2
:1030C000B78382819381019693838283DF0101C05C
:1030D000D201CD01CDB7DEB7E2E10C946B1EA0E2C8
:1030E000B0E0E5E7F8E10C945B1E69837A838B839B
:1030F0009C832D833E834F835887E9E0EE2EF12C8D
:10310000EC0EFD1ECE010196B7010E94221D8E011C
:103110000F5E1F4FCE010596B8010E94221D8A89BD
:1031200091E089278A8BC701B801AE01475E5F4FE6
:103130000E9423170E944D1CA096E6E00C94771E77
:10314000A0E2B0E0E6EAF8E10C945B1E69837A83C2
:103150008B839C832D833E834F835887F9E0EF2E2A
:10316000F12CEC0EFD1ECE010196B7010E94221D2E
:103170008E010F5E1F4FCE010596B8010E94221DE1
:10318000C701B801AE01475E5F4F0E9423170E943E
:103190004D1CA096E6E00C94771EA0E2B0E0E3EDB3
:1031A000F8E10C944F1E69837A838B839C832D8373
:1031B0003E834F835887CE010196BE01675F7F4FE4
:1031C0000E94221DCE010596BE016F5E7F4F0E94B8
:1031D000221D9985923088F089898230C8F0943018
:1031E00019F4823051F404C0843029F4923081F40F
:1031F00088EA91E0C6C0923049F420E09A858A8935
:10320000981321E02A87CE010996BBC0823049F489
:1032100020E09A858A89981321E02A8BCE01419675
:10322000B0C02D843E844F8458886D887E888F88F6
:10323000988CEE24FF248701AA24BB24650140E07A
:1032400050E060E070E0E0E0F0E0C101817090707B
:10325000892BE9F0E60CF71C081D191D9A01AB013A
:103260002A0D3B1D4C1D5D1D80E090E0A0E0B0E00C
:10327000E614F7040805190520F481E090E0A0E0C9
:10328000B0E0BA01A901480F591F6A1F7B1FAA0CA1
:10329000BB1CCC1CDD1C97FE08C081E090E0A0E0C8
:1032A000B0E0A82AB92ACA2ADB2A3196E032F10511
:1032B00049F0660C771C881C991C569447943794E7
:1032C0002794C3CFFA85EA892B893C898B859C8515
:1032D000280F391F2E5F3F4F17C0CA0181709070B1
:1032E000892B61F016950795F794E79480E090E0BC
:1032F000A0E0B0E8E82AF92A0A2B1B2B76956795FF
:10330000579547952F5F3F4F77FDE7CF0CC0440F90
:10331000551F661F771F17FD4160EE0CFF1C001F35
:10332000111F21503040403090E0590790E069076C
:1033300090E4790760F32B8F3C8FDB01CA018F7714
:103340009070A070B07080349105A105B10561F452
:1033500047FD0AC0E114F1040105110529F0405CA4
:103360005F4F6F4F7F4F40781A8EFE1711F081E04C
:103370008A8F4D8F5E8F6F8F78A383E0898FCE0108
:1033800049960E944D1CA096E2E10C946B1EA8E1A8
:10339000B0E0EDECF9E10C94571E69837A838B83DE
:1033A0009C832D833E834F835887B9E0EB2EF12C0D
:1033B000EC0EFD1ECE010196B7010E94221D8E016A
:1033C0000F5E1F4FCE010596B8010E94221D298570
:1033D000223008F47EC03989323010F4B8017CC044
:1033E0008A859A8989278A87243011F0223031F41E
:1033F000231709F06EC068EA71E06EC0343039F40A
:103400001D861E861F86188A1C861B8604C03230C5
:1034100021F484E08987B7015FC02B853C858B89C7
:103420009C89281B390B3C872B87ED84FE840F85F4
:103430001889AD88BE88CF88D88CEA14FB040C05A7
:103440001D0540F4EE0CFF1C001F111F21503040E1
:103450003C872B8720E030E040E050E080E090E0C7
:10346000A0E0B0E460E070E0EA14FB040C051D0588
:1034700040F0282B392B4A2B5B2BEA18FB080C0950
:103480001D09B695A79597958795EE0CFF1C001F13
:10349000111F6F5F7F4F6F31710531F7DA01C9017D
:1034A0008F779070A070B07080349105A105B10540
:1034B00061F427FD0AC0E114F1040105110529F0AA
:1034C000205C3F4F4F4F5F4F20782D873E874F87BF
:1034D000588BBE01675F7F4FCB010E944D1C6896E1
:1034E000EAE00C94731EA8E1B0E0E9E7FAE10C947D
:1034F0005B1E69837A838B839C832D833E834F83FA
:10350000588789E0E82EF12CEC0EFD1ECE010196C5
:10351000B7010E94221D8E010F5E1F4FCE0105963E
:10352000B8010E94221D8985823040F0898982304D
:1035300028F0C701B8010E949A1D01C08FEF68965C
:10354000E6E00C94771EA8E1B0E0E9EAFAE10C9419
:103550005B1E69837A838B839C832D833E834F8399
:10356000588789E0E82EF12CEC0EFD1ECE01019665
:10357000B7010E94221D8E010F5E1F4FCE010596DE
:10358000B8010E94221D8985823040F089898230ED
:1035900028F0C701B8010E949A1D01C081E0689619
:1035A000E6E00C94771EA8E0B0E0E9EDFAE10C94B7
:1035B000581E9B01AC0183E08983DA01C901882789
:1035C000B7FD83959927AA27BB27B82E211531056A
:1035D0004105510519F482E089833AC08823A9F096
:1035E000203080E0380780E0480780E8580729F459
:1035F00060E070E080E09FEC30C0EE24FF248701A3
:10360000E21AF30A040B150B02C079018A018EE15C
:10361000C82ED12CDC82CB82ED82FE820F831887EC
:10362000C801B7010E94FE1B01971816190684F401
:10363000082E04C0EE0CFF1C001F111F0A94D2F7C5
:10364000ED82FE820F831887C81AD90ADC82CB82EA
:10365000BA82CE0101960E944D1C2896E9E00C9496
:10366000741EACE0B0E0E7E3FBE10C945F1E6983FD
:103670007A838B839C83CE010196BE016B5F7F4F63
:103680000E94221D8D81823061F1823050F18430A0
:1036900021F48E81882351F12EC02F81388537FD8A
:1036A00020C06E812F3131051CF06623F9F023C054
:1036B0008EE190E0821B930B29853A854B855C85D2
:1036C00004C056954795379527958A95D2F7662376
:1036D000B1F050954095309521953F4F4F4F5F4F3A
:1036E0000EC020E030E040E050E009C02FEF3FEF97
:1036F0004FEF5FE704C020E030E040E050E8B90160
:10370000CA012C96E2E00C947B1EA8E0B0E0EBE846
:10371000FBE10C94571E7B018C016115710581053D
:10372000910519F482E0898360C083E089838EE18A
:10373000C82ED12CDC82CB82ED82FE820F831887CB
:10374000C801B7010E94FE1BFC013197F7FF3BC087
:10375000222733272E1B3F0B57016801022E04C07E
:10376000D694C794B794A7940A94D2F740E050E057
:1037700060E070E081E090E0A0E0B0E004C0880F7D
:10378000991FAA1FBB1F2A95D2F70197A109B1095A
:103790008E219F21A023B1230097A105B10521F01F
:1037A00041E050E060E070E04A295B296C297D2906
:1037B0004D835E836F8378878EE190E08E1B9F0B35
:1037C0009C838B8312C0309781F00E2E04C0EE0CC8
:1037D000FF1C001F111F0A94D2F7ED82FE820F8397
:1037E0001887CE1ADF0ADC82CB821A82CE010196BC
:1037F0000E944D1C2896EAE00C94731EEF92FF92F3
:103800000F931F937B018C0180E0E81680E0F8069F
:1038100081E0080780E0180788F48FEFE816F104CC
:103820000105110531F028F088E090E0A0E0B0E05B
:1038300017C080E090E0A0E0B0E012C080E0E816A1
:1038400080E0F80680E0080781E0180728F088E1AA
:1038500090E0A0E0B0E004C080E190E0A0E0B0E043
:1038600020E230E040E050E0281B390B4A0B5B0BB4
:1038700004C016950795F794E7948A95D2F7F70157
:10388000E055FE4F8081281B310941095109C901CA
:103890001F910F91FF90EF900895DF92EF92FF92AA
:1038A0000F931F93FC01E480F58006811781D1807E
:1038B0008081823048F480E090E0A0E1B0E0E82A26
:1038C000F92A0A2B1B2BA5C0843009F49FC0823033
:1038D00021F4EE24FF24870105C0E114F104010561
:1038E000110519F4E0E0F0E096C0628173819FEF6A
:1038F000623879070CF05BC022E83FEF261B370BDC
:103900002A3131052CF020E030E040E050E02AC0C0
:10391000B801A701022E04C0769567955795479583
:103920000A94D2F781E090E0A0E0B0E004C0880FF4
:10393000991FAA1FBB1F2A95D2F70197A109B109A8
:103940008E219F21A023B1230097A105B10521F06D
:1039500081E090E0A0E0B0E09A01AB01282B392B88
:103960004A2B5B2BDA01C9018F779070A070B07081
:1039700080349105A105B10539F427FF09C0205C09
:103980003F4F4F4F5F4F04C0215C3F4F4F4F5F4F42
:10399000E0E0F0E02030A0E03A07A0E04A07A0E431
:1039A0005A0710F0E1E0F0E079018A0127C06038A1
:1039B000710564F5FB01E158FF4FD801C7018F770E
:1039C0009070A070B07080349105A105B10539F4F4
:1039D000E7FE0DC080E490E0A0E0B0E004C08FE31B
:1039E00090E0A0E0B0E0E80EF91E0A1F1B1F17FFD1
:1039F00005C016950795F794E794319687E01695DC
:103A00000795F794E7948A95D1F705C0EE24FF2433
:103A10008701EFEFF0E06E2F679566276795902F8F
:103A20009F77D794DD24D7948E2F8695492F462BE8
:103A3000582F5D29B701CA011F910F91FF90EF9098
:103A4000DF900895FC01DB01408151812281622FCA
:103A50006F7770E0221F2227221F9381892F880F02
:103A6000822B282F30E0991F9927991F11969C933C
:103A7000119721153105A9F541155105610571050C
:103A800011F482E037C082E89FEF13969C938E93E7
:103A900012979A01AB0167E0220F331F441F551F95
:103AA0006A95D1F783E08C930DC0220F331F441F1A
:103AB000551F12968D919C911397019713969C9385
:103AC0008E931297203080E0380780E0480780E42A
:103AD000580758F314962D933D934D935C93179785
:103AE00008952F3F310579F44115510561057105A0
:103AF00019F484E08C93089564FF03C081E08C93F3
:103B000012C01C9210C02F57304013963C932E9336
:103B1000129783E08C9387E0440F551F661F771F31
:103B20008A95D1F7706414964D935D936D937C9351
:103B3000179708951F93DC01FB019C91923008F4C4
:103B400047C08081823008F443C0943051F411960C
:103B50001C91843099F58181682F70E0611B710997
:103B60003FC0843021F0923031F48230B9F181814C
:103B7000882389F12DC011961C9111978230F1F0A4
:103B800081811817D9F412962D913C911397828157
:103B900093818217930794F028173907BCF0149685
:103BA0008D919D910D90BC91A02D248135814681F0
:103BB0005781281739074A075B0718F4112341F08A
:103BC0000AC082179307A407B50740F4112319F020
:103BD00061E070E005C06FEF7FEF02C060E070E071
:103BE000CB011F910895629FD001739FF001829FC6
:103BF000E00DF11D649FE00DF11D929FF00D839F7C
:103C0000F00D749FF00D659FF00D9927729FB00D18
:103C1000E11DF91F639FB00DE11DF91FBD01CF012B
:103C200011240895A1E21A2EAA1BBB1BFD010DC091
:103C3000AA1FBB1FEE1FFF1FA217B307E407F5075C
:103C400020F0A21BB30BE40BF50B661F771F881F38
:103C5000991F1A9469F760957095809590959B01CE
:103C6000AC01BD01CF01089597FB092E05260ED0AA
:103C700057FD04D0D7DF0AD0001C38F4509540958A
:103C8000309521953F4F4F4F5F4F0895F6F7909530
:103C90008095709561957F4F8F4F9F4F08952F921C
:103CA0003F924F925F926F927F928F929F92AF92CC
:103CB000BF92CF92DF92EF92FF920F931F93CF9319
:103CC000DF93CDB7DEB7CA1BDB0B0FB6F894DEBFB0
:103CD0000FBECDBF09942A88398848885F846E84D6
:103CE0007D848C849B84AA84B984C884DF80EE8020
:103CF000FD800C811B81AA81B981CE0FD11D0FB629
:103D0000F894DEBF0FBECDBFED010895EE0FFF1F8B
:103D10000590F491E02D0994CF93DF93BC0182309C
:103D2000910510F462E070E0A0919003B0919103CE
:103D3000ED01E0E0F0E040E050E021C088819981B1
:103D40008617970769F48A819B81309719F09383CE
:103D5000828304C09093910380939003FE0134C04A
:103D60006817790738F44115510519F0841795073C
:103D700008F4AC01FE018A819B819C01E901209736
:103D8000E9F641155105A9F1CA01861B970B049765
:103D900008F4BA01E0E0F0E02AC08D919C911197FF
:103DA00084179507F9F46417750781F412968D91BD
:103DB0009C911397309719F09383828304C090935A
:103DC000910380939003FD0132964FC0CA01861B78
:103DD000970BFD01E80FF91F6193719302978D9383
:103DE0009C9343C0FD01828193819C01D90110976E
:103DF000A1F680918E0390918F03892B41F48091DD
:103E0000B2029091B30290938F0380938E034091FE
:103E1000B4025091B5024115510541F44DB75EB75A
:103E20008091B0029091B102481B590B20918E03F2
:103E300030918F0324173507B0F4CA01821B930B0E
:103E40008617970780F0AB014E5F5F4F8417950789
:103E500050F0420F531F50938F0340938E03F9018C
:103E60006193719302C0E0E0F0E0CF01DF91CF9168
:103E70000895CF93DF93009709F450C0EC01229787
:103E80001B821A82A0919003B0919103109709F1BF
:103E900040E050E0AC17BD0708F1BB83AA83FE01E8
:103EA00021913191E20FF31FAE17BF0779F48D9185
:103EB0009C911197280F391F2E5F3F4F398328831C
:103EC00012968D919C9113979B838A83411551057E
:103ED00071F4D0939103C093900320C012968D91FA
:103EE0009C911397AD01009711F0DC01D3CFFA013B
:103EF000D383C28321913191E20FF31FCE17DF07E5
:103F000069F488819981280F391F2E5F3F4FFA018C
:103F1000318320838A819B8193838283DF91CF9138
:103F20000895A0E0B0E0E7E9FFE10C94571EEC0132
:103F3000A880B980CA80DB80A114B104C104D10477
:103F400041F484E2A82E89EDB82E8BE5C82E87E0D7
:103F5000D82EC601B5012DE133EF41E050E00E94BB
:103F6000341E27EA31E440E050E00E94F31D7B015B
:103F70008C01C601B5012DE133EF41E050E00E9414
:103F8000341ECA01B9012CEE34EF4FEF5FEF0E94EF
:103F9000F31D6E0D7F1D801F911F97FF04C06150A0
:103FA000704080409048688379838A839B839B011B
:103FB000AC015F77B901CA01CDB7DEB7EAE00C9476
:103FC000731E0E94911F089586EB92E00E94911F3C
:103FD00008956093B6027093B7028093B8029093ED
:103FE000B9020895A0E0B0E0E8EFFFE10C94551E9F
:103FF0008C01009729F4CB010E948C1E8C01BAC061
:104000009EEFE92E9FEFF92EE00EF11E5801A60E4D
:10401000B71EAE14BF0408F4ABC08EEF882E8FEF2E
:10402000982E8A0C9B1CE701488159814617570737
:10403000B8F04530510508F49DC0CA0104978617B1
:10404000970708F497C042505040461B570BF401A5
:104050005183408379836883C5010E94391F8AC0D8
:104060006B01C41AD50AE0919003F0919103A0E08E
:10407000B0E0C0E0D0E042C0E815F905A1F520812C
:1040800031812C153D0578F1C90102968C159D05ED
:10409000A8F04E5F5F4F420F531FE70159834883DB
:1040A00022813381109729F013963C932E93129717
:1040B00061C030939103209390035CC02250304044
:1040C0002C193D0931832083109729F01396FC9316
:1040D000EE93129704C0F0939103E0939003F701DD
:1040E0007183608347C080819181C817D90708F424
:1040F000EC01DF01828193819C01F901309709F085
:10410000BBCF400F511F80918E0390918F03841776
:104110009507E9F4C617D707D0F42091B40230917F
:10412000B5022115310541F42DB73EB78091B0029B
:104130009091B102281B390BA216B306C8F4B092B5
:104140008F03A0928E03E7017983688313C0CB01AC
:104150000E948C1EEC01009759F0F70140815181BB
:10416000B8010E94FF20C8010E94391F8E0102C0C1
:1041700000E010E0C801CDB7DEB7ECE00C94711E92
:104180001F93FC0199278827BC01E89411911032F4
:10419000E9F3193010F01E30C8F31B3251F01D3214
:1041A00049F4689406C00E94C521610F711D811DEC
:1041B000911D119110531A30B0F33EF490958095F3
:1041C000709561957F4F8F4F9F4F1F91089591116B
:1041D00016C1803219F089508550D0F70895911199
:1041E000089581548A5108F4805E855A089591118A
:1041F000089581568A5108F4805285580895FB012C
:10420000DC0102C001900D9241505040D8F7089552
:10421000FB01DC010D900020E9F7119701900D9250
:104220000020E1F70895FC018191861721F0882391
:10423000D9F7992708953197CF010895FB01DC0143
:104240008D91019080190110D9F3990B0895FB010C
:10425000DC0101900D920020E1F70895FB01DC01E3
:104260004150504030F08D910190801919F4002098
:10427000B9F7881B990B0895FB01DC0141505040B0
:1042800048F001900D920020C9F701C01D924150E5
:104290005040E0F70895FC0181E090E0019006169F
:1042A00009F4CF010020D1F701970895FB01519146
:1042B0005523A9F0BF01DC014D9145174111E1F7EC
:1042C00059F4CD010190002049F04D914015411164
:1042D000C9F3FB014111EFCF81E090E00197089510
:1042E000FB019F01E8944230C4F04532B4F44A30F7
:1042F00029F497FB1EF4909581959F4F642F7727A3
:104300000E941222805D8A330CF0895D8193CB017B
:104310000097A1F716F45DE251931082C9010C9445
:104320000222FA01CF93FF93EF93223044F125321A
:1043300034F5C22FE894CA3049F497FB3EF49095C7
:104340008095709561957F4F8F4F9F4F2C2F33270E
:1043500044275527FF93EF930E94121EEF91FF9180
:10436000605D6A330CF0695D6193B901CA01605008
:1043700070408040904051F716F4CDE2C193108216
:104380008F919F91CF910C940222592F482F372F54
:10439000262F660F771F881F991F660F771F881FAC
:1043A000991F620F731F841F951F660F771F881F49
:1043B000991F0895FA01CF93FF93EF932230CCF029
:1043C0002532BCF4C22F2C2F332744275527FF93C7
:1043D000EF930E94121EEF91FF91605D6A330CF023
:1043E000695D6193B901CA0160507040804090409E
:1043F00051F710828F919F91CF910C9402229927AF
:1044000088270895DC01FC01672F71917723E1F77C
:10441000329704C07C916D9370836291AE17BF0791
:10442000C8F30895AA1BBB1B51E107C0AA1FBB1FFD
:10443000A617B70710F0A61BB70B881F991F5A9530
:10444000A9F780959095BC01CD010895F894FFCF10
:104450000D0A2B494E513D310D0A000D0A2B5354C4
:10446000574D4F443D300D0A000D0A2B53544E4119
:104470003D4164617074696373456C65637469631D
:104480000D0A000D0A2B53544F4155543D310D0A6E
:10449000000D0A2B53544155544F3D300D0A000D69
:1044A0000A202B535450494E3D303030300D0A0015
:1044B0000D0A2B4C4F53535245434F4E4E3D300D3A
:1044C0000A0007F000000000008E04DB04F3043350
:1044D000045E044404820400000000DA00DB04F3FC
:1044E00004DA00DA00DA00DA002E0000000000DA58
:1044F00000DB04F304FF00010000000000000000E6
:10450000000102020303030304040404040404047A
:10451000050505050505050505050505050505054B
:10452000060606060606060606060606060606062B
:10453000060606060606060606060606060606061B
:1045400007070707070707070707070707070707FB
:1045500007070707070707070707070707070707EB
:1045600007070707070707070707070707070707DB
:1045700007070707070707070707070707070707CB
:1045800008080808080808080808080808080808AB
:10459000080808080808080808080808080808089B
:1045A000080808080808080808080808080808088B
:1045B000080808080808080808080808080808087B
:1045C000080808080808080808080808080808086B
:1045D000080808080808080808080808080808085B
:1045E000080808080808080808080808080808084B
:1045F000080808080808080808080808080808083B
:0A46000020009203000001000000FA
:00000001FF
